:10000000CB28A0008417800484138E010C1C8E0062
:1000100023200319C62823200319C6282320C62815
:10002000A00059200C080D040319C628C020841311
:100030002008800664001C281D288C0A03198D0FD7
:100040001A288006C62820088E0601308C008D01F3
:10005000000820050E06031D08008C0A03198D0FE9
:10006000282808008F002208840020095A208413C1
:100070008F080319C628F03091000E0880389000D0
:10008000F03091030319910003198F030319C62857
:1000900049285D2003010C1820088E1F20088E08B7
:1000A00003190301900F562880063D2857280000A9
:1000B0004028FF3A84178005C6280D080C04031950
:1000C0008C0A80300C1A8D060C198D068C188D0642
:1000D0000D0D8C0D8D0DC6288F018E00FF308E0703
:1000E000031C8F07031CC62803308D00DF307A20E5
:1000F0006E288D01E83E8C008D09FC30031C83289E
:100100008C07031880288C0764008D0F80280C183A
:1001100089288C1C8D2800008D2808008E00033053
:1001200094288E000430942894000F080D02031DBB
:100130009B280E080C02043003180130031902300A
:100140001405031DFF30C628910190011030920064
:100150000D0D900D910D0E0890020F08031C0F0F4E
:1001600091020318BA280E0890070F0803180F0F02
:10017000910703108C0D8D0D920BA8280C08C62832
:100180008C098D098C0A03198D0A08008313031347
:1001900083126400080083168501083086008312EC
:1001A0000611831606118312861083168610831299
:1001B00006108316061083120130B1006400063069
:1001C00031020318E6286B21B10FDE28AA01A40131
:1001D000A501AB0164000B302B0203180329B521E4
:1001E00026088C0027088D0025088F002408912000
:1001F000031D00292608A4002708A5002B08AA0033
:100200009021AB0FEA282A080B3CAE000130B10068
:10021000640031082E02031C10296B21B10F08293C
:100220000130B10064001030310203182629B521D5
:1002300026088C0027088D008F0106308E20031DB4
:1002400023293A21DC282921B10F1229DC28630057
:100250002729AA30AD00D421A030AC00A030AF00D7
:10026000D4216430AD00D4217830AC007830AF00B8
:10027000D4210800B10164000430310203186A2956
:100280000630A2001030A0005A308E00013032201B
:1002900050308E00023032207D308E00013032200E
:1002A0005A308E000230322064308E00023032200C
:1002B000AA30AD00D4217830AC007830AF00D42122
:1002C0006430AD00D421A030AC00A030AF00D42108
:1002D000B10F3B2908000630A2001030A0008C307E
:1002E0008E000130322050308E00023032207D30BE
:1002F0008E00013032205F308E0002303220AA3072
:10030000AD00D4217830AC00A030AF00D4216430EF
:10031000AD00D421A030AC007830AF00D42108006B
:100320000630A2001030A0008C308E000130322048
:1003300078308E00023032206E308E000130322054
:1003400064308E0002303220AA30AD00D421A030BB
:10035000AC007830AF00D4216430AD00D4217830C7
:10036000AC00A030AF00D421080001308C008D011A
:10037000063084000430102001308C0006308400E8
:10038000083001200C08A8000D08A90028088C00DE
:1003900029088D000F308E008F01A420A6000D08C3
:1003A000A70001306C2008000130B00064000B3061
:1003B00030020318F4292D088C008D0106308400CA
:1003C000803010202C088C008D01063084004030D5
:1003D00010202F088C008D01063084002030102062
:0A03E0000D306C20B00FD629080084
:02400E00F53F7C
:00000001FF
